:1000000000308A005F280000FF00030E8301A60075
:100010007F08A5000A08AD008A01A50E0408A70004
:100020002008A8002108A9002208AA002308AB0084
:100030002408AC00831383128B1E20280B1933284D
:10004000270884002808A0002908A1002A08A20087
:100050002B08A3002C08A4002D088A00260E83007C
:10006000FF0E7F0E09008A11352830088100B10B80
:1000700046283230B100831685168312851E422829
:100080008512432885168316851283120B118A1157
:10009000202833308400000803195D280330A100B4
:1000A000A001A00B5128A10B50283C30A000A00BB0
:1000B000572800000000800B4E288A1181298401F6
:1000C0001F30830583161F149F141F159F110730BF
:1000D00083129F00FF30B2003230B100321032087C
:1000E0008316870083120714B21132088316870023
:1000F0008312871501308316850000308600870043
:100100008312B2003211320883168700831207115E
:100110000C309700B21032088316870083128710C4
:100120000C309D000030A10004389200FF3083168F
:1001300092001F109F141F159F151F1383121F136A
:100140009F1783169F1783121F1483160108C03947
:1001500007388100831281018B16C0308B04003078
:10016000A1001F08C73921049F001030A000A00B78
:10017000B72800001F151F19BB2883161E088312FD
:10018000AE001E08AF002F08013C03180F29FF3AEC
:10019000031DCE282E08103C03180F2932103208F8
:1001A0008316870083120714B21132088316870062
:1001B0008312871500302E02A0002F08A300023002
:1001C000031C0330A3022008A2000310200DB3007B
:1001D000230DB400B40CB30CB40CB30CB40C330842
:1001E0009B00B40C340C3039A0001D08CF3920041A
:1001F0009D009501B2113208831687008312871182
:1002000000302E02B3002F08B4000230031C03306C
:10021000B4020310340CA300330CA200B0002F086A
:10022000013C031C5A29031D19292E08EF3C031C0D
:100230005A29321032088316870083120714B2112C
:10024000320883168700831287159B012E08FF3C16
:10025000A0000130A3002F08031C2F0FA3022008C9
:10026000A2000310200DB300230DB400B40CB30C96
:10027000B40CB30CB40C33089500B40C340C303906
:10028000A0001708CF3920049700321032088316D7
:100290008700831207102E08FF3CB3000130B40022
:1002A0002F08031C2F0FB4020310340CA300330CCF
:1002B000A200B0002F08003C03187E29FF3A031D5E
:1002C00065292E08EF3C03187E292F08023C031CE9
:1002D0007E29031D6F292E08103C031C7E29321035
:1002E00032088316870083120714B211320883166E
:1002F00087008312871595019B01B0011430B3006C
:060300004928AF2863004C
:02400E00723FFF
:00000001FF
